:100000000210ADE4FFFE12014C600C0FEF70010E08
:1000100009E970F20A80EF22000122024039010052
:10002000000022023090E4FF02172502403CEFC39B
:1000300094094005EF940E4004EFB42003D38001EF
:02004000C322D9
:0E004300024CD4A120000000000200023FEE9B
:1000530002408DE709F608DFFA8046E709F208DF78
:10006300FA803E88828C83E709F0A3DFFA8032E3CB
:1000730009F608DFFA8078E309F208DFFA8070886E
:10008300828C83E309F0A3DFFA806489828A83E0A8
:10009300A3F608DFFA805889828A83E0A3F208DF97
:1000A300FA804C80D280FA80C680D4806980F28046
:1000B30033801080A680EA809A80A880DA80E2806C
:1000C300CA803389828A83ECFAE493A3C8C582C8C1
:1000D300CCC583CCF0A3C8C582C8CCC583CCDFE92B
:1000E300DEE7800D89828A83E493A3F608DFF9ECC7
:1000F300FAA9F0EDFB2289828A83ECFAE0A3C8C552
:1001030082C8CCC583CCF0A3C8C582C8CCC583CC78
:10011300DFEADEE880DB89828A83E493A3F208DFE7
:10012300F980CC88F0EF60010E4E60C388F0ED24B7
:1001330002B4040050B9F582EB2402B4040050AFBA
:1001430023234582239000A673BB010689828A83F9
:10015300E0225002E722BBFE02E32289828A83E483
:100163009322BB010CE58229F582E5833AF583E00E
:10017300225006E92582F8E622BBFE06E92582F82D
:10018300E222E58229F582E5833AF583E49322BBF3
:10019300010689828A83F0225002F722BBFE01F313
:1001A30022F8BB010DE58229F582E5833AF583E860
:1001B300F0225006E92582C8F622BBFE05E9258216
:1001C300C8F222EF8DF0A4A8F0CF8CF0A428CE8D36
:1001D300F0A42EFE22BC000BBE0029EF8DF084FF9D
:1001E300ADF022E4CCF875F008EF2FFFEE33FEEC10
:1001F30033FCEE9DEC984005FCEE9DFE0FD5F0E937
:10020300E4CEFD22EDF8F5F0EE8420D21CFEADF035
:1002130075F008EF2FFFED33FD4007985006D5F03A
:10022300F222C398FD0FD5F0EA22C5F0F8A3E02827
:10023300F0C5F0F8E582158270021583E038F022EC
:10024300A3F8E0C5F025F0F0E5821582700215836E
:10025300E0C838F0E822BB010A89828A83E0F5F01E
:10026300A3E022500687F009E71922BBFE07E3F556
:10027300F009E3192289828A83E493F5F0740193E8
:1002830022BB010A89828A83F0E5F0A3F02250069B
:10029300F709A7F01922BBFE06F3E5F009F31922CB
:1002A300F8BB0111E58229F582E5833AF583E8F08D
:1002B300E5F0A3F0225009E92582C8F608A6F0224A
:1002C300BBFE09E92582C8F2E5F008F222E88FF0C7
:1002D300A4CC8BF0A42CFCE98EF0A42CFC8AF0EDCA
:1002E300A42CFCEA8EF0A4CDA8F08BF0A42DCC387E
:1002F30025F0FDE98FF0A42CCD35F0FCEB8EF0A4B6
:10030300FEA9F0EB8FF0A4CFC5F02ECD39FEE43C6F
:10031300FCEAA42DCE35F0FDE43CFC2275F0087513
:100323008200EF2FFFEE33FECD33CDCC33CCC5822D
:1003330033C5829BED9AEC99E58298400CF582EEE9
:100343009BFEED9AFDEC99FC0FD5F0D6E4CEFBE4D1
:10035300CDFAE4CCF9A88222B800C1B90059BA0099
:100363002DEC8BF084CFCECDFCE5F0CBF97818EFF4
:100373002FFFEE33FEED33FDEC33FCEB33FB10D7F5
:1003830003994004EB99FB0FD8E5E4F9FA227818B6
:10039300EF2FFFEE33FEED33FDEC33FCC933C91011
:1003A300D7059BE99A4007EC9BFCE99AF90FD8E043
:1003B300E4C9FAE4CCFB2275F010EF2FFFEE33FE15
:1003C300ED33FDCC33CCC833C810D7079BEC9AE888
:1003D30099400AED9BFDEC9AFCE899F80FD5F0DA09
:1003E300E4CDFBE4CCFAE4C8F922EB9FF5F0EA9EF6
:1003F30042F0E99D42F0E89C45F022E8600FECC32F
:1004030013FCED13FDEE13FEEF13FFD8F122E6FC10
:1004130008E6FD08E6FE08E6FF22E6FB08E6F90823
:10042300E6FA08E6CBF8227401FF3395E0FEFDFC03
:10043300A3A3A3E0CF2FF0E582158270021583E01A
:10044300CE3EF0E582158270021583E0CD3DF0E5E6
:1004530082158270021583E0CC3CF022ECF608EDA5
:10046300F608EEF608EFF622ECF0A3EDF0A3EEF0BB
:10047300A3EFF022D083D082E493F608740193F6BD
:1004830008740293F608740393F6740473A88285C0
:1004930083F0D083D0821204A71204A71204A712F8
:1004A30004A7E473E493A3C583C5F0C583C8C582D9
:1004B300C8F0A3C583C5F0C583C8C582C822D0834D
:1004C300D082F8E4937012740193700DA3A393F890
:1004D300740193F5828883E4737402936860EFA3D5
:1004E300A3A380DFD083D082F8E4937012740193C6
:1004F300700DA3A393F8740193F5828883E4737456
:100503000293B5F0067403936860E9A3A3A3A380E1
:10051300D8D083D082E4937012740193700DA3A397
:1005230093F8740193F5828883E4737402936C7077
:10053300127403936D700C7404936E7006740593B8
:100543006F60DDA3A3A3A3A3A380CA8A838982E4E4
:1005530073E3F5F009E208B5F06BDFF58067E3F5C7
:10056300F009E608B5F05EDFF5805A87F009E60882
:10057300B5F052DFF6804E87F009E208B5F046DFAA
:10058300F6804288828C8387F009E0A3B5F036DFDA
:10059300F6803288828C8387F009E493A3B5F02533
:1005A300DFF5802188828C83E3F5F009E0A3B5F0C1
:1005B30014DFF5801088828C83E3F5F009E493A3BC
:1005C300B5F002DFF4020683808780E9809080D44F
:1005D300803E8015806E807E809D80B7808D80A355
:1005E30080518074803C02068F89828A83ECFAE40E
:1005F30093F5F0A3C8C582C8CCC583CCE493A3C844
:10060300C582C8CCC583CCB5F076DFE3DEE180706C
:1006130089828A83E493F5F0A3E208B5F062DFF4FC
:10062300805E89828A83E0F5F0A3E608B5F051DFA6
:10063300F5804D89828A83E0F5F0A3E208B5F040A6
:10064300DFF5803C89828A83E493F5F0A3E608B55D
:10065300F02EDFF4802A8002805789828A83ECFAA5
:10066300E493F5F0A3C8C582C8CCC583CCE0A3C886
:10067300C582C8CCC583CCB5F006DFE4DEE28000DA
:100683007FFFB5F0020F2240027F012289828A8315
:10069300ECFAE0F5F0A3C8C582C8CCC583CCE0A3CF
:1006A300C8C582C8CCC583CCB5F0D5DFE5DEE38011
:1006B300CF89828A83ECFAE0F5F0A3C8C582C8CC5F
:1006C300C583CCE493A3C8C582C8CCC583CCB5F09D
:1006D300AFDFE4DEE280A988F0EF60010E4E60AB8D
:1006E300ED2402B404005098F582EB2402B4040014
:1006F300508E23234582239005CB73EF4E6012EF78
:1007030060010EEDBB010B89828A83F0A3DFFCDE5F
:10071300FA2289F05007F709DFFCA9F022BBFEFC9F
:10072300F309DFFCA9F022C3E49FFFE49EFEE49DEE
:10073300FDE49CFC22F8E0FBA3A3E0F925F0F0E53F
:1007430082158270021583E0FA38F022EBF0A3EAF7
:10075300F0A3E9F022E52524A4F582E4340EF58321
:10076300E0052522900EA1300803900EA4E475F055
:100773000112073802014C2001E97F2ED2018018B3
:10078300EF540F2490D43440D4FF30050BEF24BF33
:10079300B41A0050032461FFE526600215260529DB
:1007A300E5297002052830080E900EA1E475F001CA
:1007B300120738EF0201920211987403D2088003E2
:1007C300E4C208F525900EA112074FE4F526F5289B
:1007D300F529E52660077F2012079B80F57527FF23
:1007E300C202C201C203C204C206C207C20912077F
:1007F30067FF700D3008057F001207ACAF29AE28E4
:1008030022B4255FC2D5C205120767FF24D0B40AFC
:1008130000501A75F00A782630D50508B6FF010690
:10082300C6A426F620D5047002D20480D924CFB4FE
:100833001A00EF5004C2E5D2050209ADD20280C608
:10084300D20180C0D20380BCD2D580BAD20680B494
:100853007F2012079B2003077401B5260040F11285
:100863000758FF12079B0207D5D209D207809512BA
:100873000758FB120758FA120758F94A4B700679C2
:100883007E7A0A7BFF20032EE526602A7E008E8275
:1008930075830012016560060EEE652770F0C2D500
:1008A300EBC0E0EAC0E0E9C0E0EE1209F4D0E0F901
:1008B300D0E0FAD0E0FB12014CFF60AAEBC0E0EA03
:1008C300C0E0E9C0E012079BD0E02401F9D0E03496
:1008D30000FAD0E0FBE5270460DCD527D980877BCD
:1008E300FF7A0979F0D203809C791080027908C2DB
:1008F30007C2098008D2D5790A8004790AC2D5E5EE
:1009030027047002F527E4FAFDFEFF120758FC7B6B
:1009130008200213120758FD7B1030010A120758F2
:10092300FE120758FF7B20EC3382D592D55013C3B8
:10093300E43001069FFFE49EFEE42002039DFDE4F4
:100943009CFCE4CBF8C202EC700CCFCECDCCE824F7
:10095300F8F870F38017C3EF33FFEE33FEED33FD8A
:10096300EC33FCEB33FB994002FB0FD8E9EB30028D
:1009730005F8D0E0C448B202C0E00AEC4D4E4F780F
:10098300207B0070C2EAB5270040BCC0E01209F624
:10099300D0F0D0E0200204C4C0E0C4B202C0F01220
:1009A3000784D0F0D5F0EB0207D51204C1087253C7
:1009B30008EC5808434C083F4208F04F08F8440835
:1009C300F84908584308FE5508E24608E24508E29C
:1009D300470A9E5008472D084B2E086E2B084F23BD
:1009E300086C200A872A080748000008663F3F3F33
:1009F30000790AA2D5200414300609B910020404B0
:100A0300B9080104A2D5200702500104200368920B
:100A130003B526005034C0E07F203004197F30A294
:100A23000372077206500F120A4DC203C207C206B1
:100A3300C2097F30800F300603E9C0E012079B3004
:100A43000603D0E0F9D0E0B526CC3006177F30B9E5
:100A5300100C12079B7F583005077F788003B90875
:100A63000312079B3003057F2D02079B7F2020097C
:100A7300F87F2B2007F322920380CF286E756C6CCE
:100A83002900D2021207583002F8C202782630D564
:100A93000108F60208072D5043495812075824034A
:100AA300B405004001E4900A999312078C743A123A
:100AB300078CD2047526040208EC31302F32332F11
:100AC30030392031363A33373A3531000D0A000DCB
:100AD3000A496E69742E2E2E000D0A253035754B8A
:100AE30020464C41534820546F74616C0D0A000931
:100AF300253035754B20464C415348204D656D6F6D
:100B030072792025640D0A000D0A253035754B20B6
:100B13004652414D0D0A002A2A4572726F722120F6
:100B230043616E6E6F7420636F6E6E6563742074C1
:100B33006F20434F4D00436F6E6E65637465642091
:100B4300746F20434F4D002A2A4572726F72212021
:100B53004E6F2064657669636520666F7220434F2C
:100B63004D002A2A4572726F722120556E72656399
:100B73006F676E697A656420726573706F6E7365F3
:100B83002022253032582220666F7220434F4D00B9
:100B93002028536174656C6C6974652900202845AD
:100BA300746865726E6574290054696D6577617642
:100BB30065204453502D44333030450D0A46697245
:100BC3006D776172653A20002052657620332E36A8
:100BD3000D0A53657269616C204E756D6265723AD8
:100BE3002000252E3573000D0A00000000205374E9
:100BF3006172742E2E2E0D0A0D0A004453502049A3
:100C03006E697469616C697A696E672E2E2E0D0A9E
:100C13000074656D7000766F6C7473007570746921
:100C23006D6500636F6D316F757400636F6D326F47
:100C3300757400737461747573006C6576656C000C
:100C43006761696E00766F6C3100766F6C32006697
:100C5300726571007265736574000D0A4453502008
:100C63004F66666C696E652E2E2E0D0A000D0A44C2
:100C73005350204F6E6C696E652E2E2E0025642016
:100C83006442205665722025642025630020256474
:100C930020487A0020454300205A50002048540041
:100CA30020505000203142002032420020334200C5
:100CB3002050430020535500466163746F72792EB0
:100CC30000427974653A202530325820205B256C28
:100CD300755D0D0A00476F6F64203A2047756167A1
:100CE300653A2025753A2575202D3E200046696C0E
:100CF3007465726564202D3E2000426164203A20B1
:100D0300005061636B65743A2025303258202530DA
:100D13003258202530325820253032580D0A0044ED
:100D2300697361626C6564204453502E2E2E0D0A44
:100D3300005772697465204661696C7572650D0AA6
:100D4300002E004661696C202530356C580D0A0071
:100D530069666C6F77732575003D256C750D0053BF
:100D630061742052656164204572726F720D0A00CE
:100D73004D452052656164204572726F720D0A0001
:100D8300FF0ABDFF0ACFFF0C57FF0D34900E11EB86
:100D9300F0A3EAF0A3E9F0900E11E0FBA3E0FAA3BD
:100DA300E0F912014CFF12002E500C900E12E47564
:100DB300F00112022D80E0D201900E11E0FBA3E0BE
:100DC300FAA3E0F912014CFF642B6004EFB42D1D6C
:100DD300900E11E0FBA3E475F001120243A9F0FAAF
:100DE30012014C642D6003D38001C39201900E1451
:100DF30012049000000000900E11E0FBA3E0FAA3A0
:100E0300E0F912014CFF1211BF5068E47F0AFEFDA6
:100E1300FC900E14E0F8A3E0F9A3E0FAA3E0FB12C0
:100E230002D0C8ECC8EDC0E0EEC0E0EFC0E0900E29
:100E330011E0FBA3E0FAA3E0F912014CFF3395E0C4
:100E4300FEEF24D0FFEE34FFFEE4FCFDD0E0FBD048
:100E5300E0FAD0E0F9EB2FFFEA3EFEED39FDEC3886
:100E6300FC900E1412046B900E12E475F001120242
:100E73002D8084300110900E14E0FCA3E0FDA3E06C
:100E8300FEA3E0FF8011900E14E0FCA3E0FDA3E0BD
:100E9300FEA3E0FF12072A22900E11EBF0A3EAF063
:100EA300A3E9F0900E11E0FBA3E0FAA3E0F912012D
:100EB3004CFF12002E500C900E12E475F00112023A
:100EC3002D80E0D201900E11E0FBA3E0FAA3E0F93C
:100ED30012014CFF642B6004EFB42D1D900E11E042
:100EE300FBA3E475F001120243A9F0FA12014C646A
:100EF3002D6003D38001C39201E4900E14F0A3F09C
:100F0300900E11E0FBA3E0FAA3E0F912014CFF12EB
:100F130011BF5042900E11E0FBA3E0FAA3E0F912D7
:100F2300014CFF3395E0FEEF24D0FBEE34FFFA9043
:100F33000E14E0FEA3E0FF7C007D0A1201C6EF2B36
:100F4300FFEE3A900E14F0A3EFF0900E12E475F05A
:100F53000112022D80AA30010A900E14E0FEA3E0D4
:100F6300FF800F900E14E0FEA3E0FFC3E49FFFE4B5
:100F73009EFE22434F4D003A2042617564200033A8
:100F830030300036303000313230300032343030DF
:100F930000343830300039363030003139323030B7
:100FA30000333834303000353736303000253032B6
:100FB300582064656661756C740020205B253032AF
:100FC300585D000D0A00526570726F6772616D693A
:100FD3006E672E2E2E20202530366C5800203D20A3
:100FE3005B2530325825303258253032585D0D0A92
:100FF3000043616E6E6F7420726570726F67726109
:101003006D2E2020496E76616C6964206461746181
:101013002066696C652E205B2530325820253032DE
:101023005820253032585D0D0A00023341E493A362
:10103300F8E493A34003F68001F208DFF48029E487
:1010430093A3F85407240CC8C333C4540F4420C8D3
:10105300834004F456800146F6DFE4800B0102046A
:1010630008102040809010B9E47E019360BCA3FF78
:10107300543F30E509541FFEE493A360010ECF549F
:10108300C025E060A840B8E493A3FAE493A3F8E48E
:1010930093A3C8C582C8CAC583CAF0A3C8C582C8FA
:1010A300CAC583CADFE9DEE780BE787EE4F6D8FDF1
:1010B300758157021068C1A3C1A400C11FC1264195
:1010C300000000021E0000021A0000021C000001C2
:1010D3003000014000022D0000410BD000410C4BB9
:1010E300004109F8004209F60000410BF100C11B61
:1010F30007440001C200000008C10BC10CC10F412D
:101103000F3A00C122C1A1410F0E00410F0C014152
:101113000F0D01410F1001410F1101410F1201C1C8
:1011230096C197C198C11AC113C114C115900E8BF2
:10113300EBF0A3EAF0A3E9F0E4900E93F0A3F090B0
:101143000E9174FFF5F012024345F0603C900E8E51
:10115300E0FBA3E0FAA3E0F912014CFF900E8BE051
:10116300FBA3E0FAA3E0F9900E93E475F0011202F9
:101173004385F082F583EF1201A4EF60C2900E8FD6
:10118300E475F00112022D80B6900E8BE0FBA3E014
:10119300FAA3E0F922EFB40A07740D1211A3740A3B
:1011A300309811A899B8130CC2983098FDA899C229
:1011B30098B811F63099FDC299F59922EFC394308E
:1011C3004007EF943A50028001C32212010002EF5C
:1011D300020140C41004800000010203010600FF65
:1011E3000901A101150026FF007508954009018139
:1011F30002954009019102C01B09026B0003010023
:101203008032080B000202020100090400000102FF
:101213000201000524001001052401010104240238
:1012230006052406000107058103400001090401A6
:1012330000020A00000007058202400000070502C1
:10124300024000000904020002030000000921110A
:10125300010001221B00070583034000010705036A
:10126300034000011C0309040908090C09100914AF
:101273000918091C090C09240928092C0930093407
:101283003203540049004D00450057004100560009
:101293004500200054004500430048004E004F0025
:1012A3004C004F0047005900200049004E00430006
:1012B3002E0014034400530050002D00440033005B
:1012C3003000300045000A033000300030003100A8
:1012D3001267128312B512C991CEE4900DFAF0E4AD
:1012E300900DF9F0900DF9E0FFC39403400261CF34
:1012F300F1F6123463900EAA120490000000017FED
:101303009012382C1256B9120026900DF8EFF09077
:101313000DF7E01204C1135841134343134A441316
:101323004A48133849135180134A8D13518E13635E
:10133300FF00001363900DFBE4F0A37480F080279B
:10134300900DFB74018013900DFB7402800C900DC3
:10135300FB74048005900DFB7408F0A3E4F0800790
:10136300E4900DFBF0A3F0D3900DFCE09400900DFE
:10137300FBE094004012900DF9E0FFF1E4900DF9C9
:10138300E0FFF1F67F0171F1900DFB12568BFD2505
:10139300E02426F582E4340F123032ED125647E48E
:1013A300F0A3F0EDD39400401BED25E02424F58257
:1013B300E4340FF58312568B125647EE8FF0120268
:1013C3002D1D80DF900DF9E004F041E791CE900DE3
:1013D300FAE004F0C39402500C900F2EE07002A3C5
:1013E300E0700241E222B139E4FF71F5E4FF71F5E7
:1013F300E4FF30F9FDC2FF8FA330FFFD22900BD233
:10140300E0FDE4FF9110900BD2E0FDE4FF900E9A13
:10141300EFF0A3EDF0900E9AE0FEF12C7002FF22A4
:1014230091CE900E9BE0C39425400A74322EB1EE08
:101433007418F08005B1E8747AF053A1CF75A27ADD
:10144300E4900E9CF0900E9AE0FF71E9900E9AE002
:10145300FFB1397FA371F5B124900E9BE0FF71F5C5
:10146300B124F11B900E9BEFF091CEE07003125567
:10147300E4900E9BE070031255E4900E9BE0600332
:10148300B4A40C900E9CE004F0E0C3940540B69025
:101493000E9BE0FF22900E9DEFF0E0FEF12C700218
:1014A300FF2291CEAF0671E9900E9DE0FFB13900A6
:1014B300000000007FA471F5F11B800F53903B43A4
:1014C300A03DD2954390447F0671F553903B43A0D2
:1014D3003DD29522900B4DE0FD7F0191E7900B4D9E
:1014E300E0FD7F01900E91EFF0A3EDF0900E91F1EE
:1014F3002A602D91CEB1397F5B71F5900E91B1EBDE
:10150300E0D394184004B124B124900E92E0FF91EB
:10151300CC900E91B1EBE0D394184004B124B124E4
:1015230022E4FFFE000FBF00010EBE03F7BFE8F485
:1015330022900DF7E0FF91CEEF146007047006C20E
:10154300A48002C2A080DA7B01900E9E7401F0FF9A
:10155300B1937B017A0B7954900E9E7404F07F0152
:10156300B1937B017A0B7954900E9E7404F07F0142
:10157300B1937B017A0B7954900E9E7404F07F0132
:10158300B1937B017A0B7954900E9E7404F07F0122
:10159300900E9AF1EA900E9AF12A604691CEB139F3
:1015A3007F5AB1E6E0D394184002B1247F01B1E63B
:1015B300E0D394184002B124900E9EE0801D900E5B
:1015C3009EE0FF14F0EF6018B1E8E0D394184002F6
:1015D300B124900E9B12308212014CFF71F580DE14
:1015E30091CE2271F5900E9AE02432F582E4340F05
:1015F300F5832291CE53A1CF75A218E4900DF8F094
:10160300E4900DF7F0123463B1347FA5F119900D16
:10161300F9EFF0900DF7E0FF24CEF582E4340BF5FB
:10162300837401F074CE2FF12E6019B134900DF94B
:10163300E04401F07FAA71F50000000000900DF96D
:10164300E0FF71F5900DF7B1EB7418F0900DF7E032
:1016530004F0E0C3940240AD91CE900DF8E004F0A5
:10166300C39402500A900BCEE07004A3E060912271
:1016730091CE4390447F0571F51256B9BFFF04C262
:1016830023801A91BF439044900DF7E054F9F0542E
:101693007FF07F0171F5900DF7E0FF71F581CE903A
:1016A3000E79F1ED74CE2FF12E7003FEFF2291CE51
:1016B300B1397F5571F57F01F119900E7DEFF0D3AC
:1016C30094004048E4A3F0125729FEC39F502C9086
:1016D3000E7CE0FFEEC39F5022F11B900E79E0FBDE
:1016E300A3E0FAA3E0F9900E7EE0F582758300EFA4
:1016F3001201A4900E7EE004F080CC125729C39F00
:10170300500AF11B900E7EE004F080EF91CE900E14
:101713007DE0FF7E002271F5E4FF000FEFB496FA3F
:10172300E4FF71F5AFA322E0FF24CEF582E4340B8E
:10173300F583E02274CE2FF12E7002FF2291CEB1F9
:10174300397FA571F5F11B81CE900E91EEF0A3F1D7
:10175300EA302332A3E07002A3E0602A91BF4390F2
:1017630044900E91E0FCA3E0FD7F0212401E900E18
:1017730096125681600E900E9312308212014CFF26
:1017830071F580EA91CE22900E8BEFF0A3EDF0A3DA
:10179300EBF0900E8BF12A6037F137900E8EEFF05D
:1017A300900E8BE0FFB139900E8EE0FF900E8CE02F
:1017B300F4FEEF5EFF900E8EF0900E8DE04FA3F0DF
:1017C3007FAA71F50000000000900E8EE0FF91CC1F
:1017D300227F03F1E47F03F1F67F0171F5E4FF61FA
:1017E300F5F1F67F5061F5EFF0A3EBF0A3EAF0A378
:1017F300E9F02253903B43A03DD295EF14601114BE
:101803006012146013146014240470134390842230
:10181300439080224390C02243904022439044222D
:10182300900E8E12046B900E8EE0FCA3E0FDA3E0FD
:10183300FEA3E0FF900E9312046B7F03900E92EFD2
:10184300F01217F600000000007F061213F5900E49
:1018530092E0FF1217F60000000000A3E0FCA3E0F3
:10186300FDA3E0FEA3E0FF900EAA12046B7F2012FB
:10187300382C53903B43A03DD295123463900E9283
:10188300E0FF1236A1EF20E0F4227E007A0B798A82
:1018930012556A7A0B794A12556A7F107D00123706
:1018A300E41206FE7E007F107D001237EB1206FE67
:1018B300E4782FF6900C06120490FFFFFFFF900BC5
:1018C300CA120490FFFFFFFF783412047700000070
:1018D30000783812047700000000E4900B34F0A382
:1018E300F07BFF7A0A79D2D125D1177FFF7833EFC6
:1018F300F6F1C678437602F1FCEE1241B0F1A3741F
:101903000AF0A374DCF0D1101207BDD110D125D198
:1019130010F1DC12358AE4F52AF1A4740AF0A374F9
:10192300F2F0E52A25E02426F582E4340FF583124C
:1019330041ABF0E52A2401FEE433A3F0A3CEF0D1BA
:10194300101207BDD110D125D110F1DC052AE52AEB
:10195300C3940340C412358A122005900EA7E4F005
:10196300A3EFF1A3740BF0A3740BF0D1101207BD16
:10197300D110D125D110F1DC122F3F900BE51204C9
:101983009000000000900BE1120490000000009012
:101993000BED12049000000000900B5074FEF01247
:1019A300313B12358AC290123472C21DC21CD282DC
:1019B300900B6574FFF01255DBE4F52BE4F52A1266
:1019C3005721BFFF09125721EFF460058000752AE4
:1019D30001E52A701674CE252BF582E4340BF583CA
:1019E300E07005752A028003752A03E52A14601244
:1019F30014601714601C240370317BFF7A0B791A6F
:101A030080277BFF7A0B7939801F7BFF7A0B794A1A
:101A13008017F1A4740BF0A37465F0A3E4F0A3E5BD
:101A23002CF0D1101207BDD110D125E52B2432FFA4
:101A3300123690E52B14600B0470107BFF7A0B7940
:101A43009380067BFF7A0B79A0D1257BFF7A0A79F5
:101A5300CFD125052BE52BD39401500221BF900B49
:101A6300DFE0FF1232E9AD077F01D1EF121400125C
:101A73001400AD077F02D1EF7D257F01121410AD55
:101A8300077F03D1EF7BFF7A0B79ACD125900D83D0
:101A9300D11A7BFF7A0B79CBD125F1A4740BF074A7
:101AA300E51255F2A3740BF0A37438F0D1101207AA
:101AB300BDD110D1257A0B79EA1235857A0B79F0ED
:101AC3001235853082091254F27A0B79FEF1F51240
:101AD300358A12313B121409D1057DFF1238A878DB
:101AE3003C120411783412571A5031783C12041105
:101AF300EF2419F1AE783412045F7841E6FE08E66C
:101B0300FF7C007D0B1201C6900BDBEEF0A3EFF020
:101B13007831E6FF08E6A3CFF0A3EFF0783C120498
:101B230011783812571A400281E4783C120411EFFD
:101B330024F4FFEE3401F1B1783812045F784006E3
:101B4300E6C394024060E4F6783006900BED12236E
:101B5300042401F1AE900BED12046B900B52E030B4
:101B6300E408782E06E6187001061257124003E0C7
:101B730004F0900C4BE0D394004010E004F0D394B5
:101B83000A40087843E654FEF6E4F030261290004B
:101B930000E0D394004005E014F0800AC2268006DA
:101BA300900000740AF0309104C2918002D29190A7
:101BB3000B52E020E40281C6900B8AE030E10281FF
:101BC300C69009F8E0FF04F0EF1204C11C0C011CDD
:101BD30017021C22031C2D041C54051C38061C541C
:101BE300081C470A1C540B1C620C1C540E1C54107A
:101BF3001C54121C47141C54151C62161C6F171C12
:101C03007C181C891B00001C9D7BFF7A0C791490A7
:101C13000BDD807B7BFF7A0C7919900BDB80707B6B
:101C2300FF7A0C791F900BED80147BFF7A0C7926D9
:101C3300900BE180097BFF7A0C792E900BE5122340
:101C430004FF804E7A0C7936900B521255A6FE8013
:101C5300417BFF7A0C793D900B4E1256B080337A5C
:101C63000C7943900BD11256CAFE80267A0C794820
:101C7300900BD31256CAFE80197A0C794D900BD46F
:101C83001255A6FE800C7BFF7A0C7952900B34120E
:101C930056B012421712413880299009F8E0C394D4
:101CA3001C4002E4F09009F61240E69009F7E024A4
:101CB30008F09009F6E03400F0C3E094204004E417
:101CC300F0A3F0D3782EE694B418E694004024E40D
:101CD300F608F612554E7B107D107F0112178A808D
:101CE30012D1107DFF1225E6D110F1B9D1057DFF88
:101CF3001238A87933E778436670051257124038D3
:101D0300900BD0E0FFD394004025EF75F00684AF2D
:101D1300F07401A807088002C333D8FCFFF1C69012
:101D23000BD0E0C3943C4010E4F07833F68009789C
:101D330043E67833F6FFF1C6D1057DFF1238A8D10B
:101D430010F1B91232B8400241DB1231178F2AE584
:101D53002AC394005002C104900A01E52AF0E4A3C7
:101D6300F078F97C097D017B017A0979FAFE7F0716
:101D73001201269009FFE52AF0E4A3F0D110D12542
:101D830078FB7C097D01900D89E412561A93F97E44
:101D9300007F051206DAEF600241DB900D891256CF
:101DA3001A93F9900E18120490000000017F01129B
:101DB30041387F007E007D047C00112312422D9068
:101DC3000BF6E4F0A3740CF0900BF4E4F0A3740CA2
:101DD300F0900BF8E4F0A3740EF0900BFEE4F0A384
:101DE3007480F0900BFCE4F0A37480F0E4A3F0A300
:101DF300F0A3F074831255F2A3742CF0123F234125
:101E0300DB227B017A0A79017DFF1228127B017A9A
:101E13000A790122900D86E493FB740193FA74020C
:101E230093F9900EA3EBF0A3EAF0A3E9F012563B6B
:101E3300EA494B6019900EA3A3A3E0120003900E8E
:101E4300A6EEF0FCA3EFF0FD12563B123622E5C9D5
:101E530020E602C1E7900B8EE0FF900B63E06F601A
:101E630002C1E7900EA6E51CF0A3E51DF0D394098B
:101E7300E51C94004009900EA6E4F0A37409F0E475
:101E8300900B64F0D3900EA7E09400900EA6E0941C
:101E9300004051900B4CE04401F07B017A0B7959DF
:101EA300900EA7E0FD1235D4900EA7E0900B64F0DE
:101EB300C3900EA7E0940A900EA6E094005017E496
:101EC30075F001120243FE745925F0F582740B3E3E
:101ED300F583E4F080DA900B63E004F0D3947F4061
:101EE300037401F0900B4CE054FEF022900E8BEF44
:101EF300F0A3EDF07BFF7A0F7976125669E0243078
:101F0300FF1236907BFF7A0F797AD125900E8CE001
:101F13001204C11F35011F3D021F45041F4D091F38
:101F230055121F5D251F654B1F6D961F75E1000040
:101F33001F7D7BFF7A0F7982804D7BFF7A0F798635
:101F430080457BFF7A0F798A803D7BFF7A0F798FFB
:101F530080357BFF7A0F7994802D7BFF7A0F7999F7
:101F630080257BFF7A0F799E801D7BFF7A0F79A4F2
:101F730080157BFF7A0F79AA800DF1A4740FF0749A
:101F8300B0122EC4125517D125F1A4740FF074BDED
:101F9300122EC4125517D1257BFF7A0F79C6C1259E
:101FA300F0900EA474FFF0A3222404FFE43EFEE4A9
:101FB3003DFDE43CFC227DFF1242487B007A007920
:101FC30000C12553903B43A03DD29553A1CF75A2A9
:101FD3007FC2A51213F5D2A52212014C6013120180
:101FE3004CFF122CA25005122ED480F212361A8006
:101FF300E8227BFFD125C21D22900F2AE0FEA3E039
:10200300FF227F082023027F00227F007E01900EA3
:10201300961217EDE4900E9BF0A3F030230A900E76
:1020230099E07002A3E07004E4FEFF221214CE4391
:102033009044AD07AC067F0312401E900E991256D2
:1020430081601D120026900E96123082EF120192CB
:10205300900E9CE004F07006900E9BE004F080DB91
:102063001214CE900E9BE0FEA3E0FF22900DFFEB37
:10207300B1DEA351E412014C900E05F0900DFF5117
:10208300E412014CFF6042640D603E900E0251E485
:1020930012014CFFD394004030900BF1E0941350A5
:1020A30028900DFF51E412014CFE900BF1E0FD046A
:1020B300F0741F2D125633EEF0900E15EFF01256FA
:1020C3009E51E4EF12019280B3900BF1E0700DE0AA
:1020D300FF04F0741F2F1256337420F0900BF1E0BD
:1020E300D3941340037413F0900BF1E0241F1256A2
:1020F30033E4F0900E05E0D39400400C900DFF51B3
:10210300E412014C640D600E900DFF51E412014C7A
:10211300640A600241B8E4900BF1F0900E0251E4BE
:1021230012014C900E15F0900DFF51E412569E5182
:10213300E4EF1201921255CC900E0651E412014CB9
:10214300FF600C643D600812562B12022D80E9EFEC
:10215300643D600241B8900E06E0FBA3E475F00114
:10216300120243A9F0FAE4120192900E0651E4120E
:10217300014CB4200812562B12022D80ED120D8F44
:10218300900E0B12046B1255CC900E0651E4120103
:102193004CB4200812562B12022D80ED120E9B9088
:1021A3000E09EEF0A3EFF0C3EE9420506D12562308
:1021B3007803CEC313CE13D8F9900E991254CF04DB
:1021C300F01111900E09E0FAA3E0FB12420F088010
:1021D30002C333D8FC900E10F0900E0B7104FFEC89
:1021E3004D4E4F700BA3E0FFA3E0F4FEEF5E800AB9
:1021F300900E0FE0FFA3E0FEEF4E900E0FF0EBAE5C
:10220300027803CEC313CE13D8F9900E961254CF8F
:1022130004F012174C900E09804A1256238EF012C6
:1022230004E7226C20002274200122416001224A2B
:1022330060022252600322646004000022B8900E00
:102243000E122F20F0806E900E0E122F2F80667FBD
:1022530001123EF17F02123EF112374512347280B1
:1022630054900E0D1240E6804C7E007F147DFF805B
:10227300067E007F147D007B017A0B791F1206FE18
:10228300E4900E09F0A3F0125623FFC3EE9404501A
:1022930024E42FFFEE3402FE7A0B791F1237BE744B
:1022A30014F012174C900E0AE02414F0900E09E07B
:1022B3003400F080D2900E0251E412014CFF900DD5
:1022C300FF51E48F82758300E40201A4F0A3EFF0D1
:1022D300900E78E0FBA3E0FAA3E0F91207BD900E9D
:1022E30078E0FBA3E0FAA3E0F922900B96E0FCA3CD
:1022F300E0FDA3E0FEA3E0FF900E7B12046B900EC3
:102303007BE0FCA3E0FDA3E0FEA3E022900E8B1292
:10231300046B900E8FEBB1DE121FA4740FF0A37445
:10232300C9F0900E8B710412420012567051E412E0
:1023330056697104FF78101203FE900E9CEFF09023
:102343000E8B7104FF78081203FE900E9DEFF09040
:102353000E8EE0900E9E121FA3740FF0A374E0F094
:10236300900E9C122EC9900E9D125582F0900E9ED7
:1023730012559CF0900E8F51E412567051E4125690
:10238300697104123FE7122CFB740EF0A37492F0F0
:10239300A37403122FDF900E92E0FF6402602B12EE
:1023A3001FA4740FF0A374F4F0A3E4F0A3EFF09070
:1023B3000E93125582F0900E9412559CF0900E8F4E
:1023C30051E412567051E4021E25E4FFE4FE000EB0
:1023D300EEB4FFFA0FEFB4FFF312358A900E9CE0D0
:1023E300FFA3E0FDA3E0FB02F800900E91EBB1DE4A
:1023F300A351E474FFF5F0120284900E9451E4901B
:10240300000274FFF5F01202A3900E9151E4124200
:10241300FDEF4E6012900E949178C9B1DB900E914E
:1024230051E4B12D7F0122900E9151E4124313EF39
:102433004E6015900E949178900E9AC9B1DE900E6D
:102443009151E491807F0122900E9151E412434017
:10245300EF4E6015900E949178900E9AC9B1DE906C
:102463000E9151E4F1957F01227F0022FFFE900B34
:1024730090FCE0F8A3E0F9A3E0FAA3E022900E9722
:10248300EBB1DE900E9751E4F1DC5401C454F01229
:102493005576C975F0001255FC51E4C003C002C063
:1024A30001120259FDACF0900E9751E4F1E27E0067
:1024B300543F7806C333CE33CED8F91256F2D00147
:1024C300D002D0031255F951E4C003C002C0011277
:1024D3000259FF900E9751E4F1F5D001D002D003D9
:1024E300F1EE900E9751E4F1DC543EFFE4C313FE8A
:1024F300EF13FF900E9A51E412553DC003C002C082
:1025030001120259FDACF0900E9751E4F1E87E0000
:10251300543F7805C333CE33CED8F91256F2D001E7
:10252300D002D003EE8FF0020284900E97EBB1DE5F
:10253300900E9751E4F1E27E00547F7806C333CEC8
:1025430033CED8F9FF900E9A51E41255F951E4C0F5
:1025530003C002C001120259FF900E9751E4F1F536
:10256300D001D002D003F1EE900E9751E4F1E27E58
:102573000054807807CEC313CE13D8F9FF900E9A78
:1025830051E412553DC003C002C001120259FD902F
:102593000E9751E4F1DC25E0FFE43345F0FEED4F07
:1025A300FFD001D002D003EE8FF0120284125577D0
:1025B300125547C003C002C001120259FD900E9785
:1025C30051E4F1E8540325E045F0FFEDD001D002DA
:1025D300D003CF8FF0020284900E9AF0A3EAF0A307
:1025E300E9F022900DF7EBB1DEA3EDF0E4A3F07F69
:1025F30001121737900DFEEFF0BFFF087BFF7A0D36
:102603007973E13E900DFEE0FF7002E141EF541853
:1026130064086002E14F900DF751E41242A07F017C
:102623001216A2900DFCEFF0E0FFD394005002E1EC
:1026330030900DF751E48F82F18E900BF1E0D3943B
:10264300004007E4900DFDF0C1DDE4900DFDF012B4
:1026530056FAFDC39F4002E130900DF751E48D829D
:10266300758300120165900DFEF054F0FEBEF01765
:10267300900E15EFF0F150900DFCEFF0900DFEE091
:1026830064F66003125702900DFEE0240CB40B00B5
:102693004002E12890269E12565E7302271C0227F1
:1026A300140226C40226DD0226520226520226D333
:1026B3000226C90226520226520226BF1257028060
:1026C3008E12554E8089E4782DF608F6D290C152C9
:1026D300E4782DF608F6C290C1521256FAFEC3EF03
:1026E3009E900DFCF0900DF751E4EEFF7E00E92F74
:1026F300F9EE3AFA900E027401F0A3740DF0A3748C
:10270300FCF0116F900DFDE0FF900DFCE02FF0C188
:1027130052900B52E044028006900B52E054FDF0BD
:10272300123745C152900DFDE004F0C152900DFCEB
:10273300E0D394004008900DF751E4121E25900D4C
:10274300FBE004F0E0C3940A5002A1F222900E11C0
:10275300EBB1DE900E15E014F0AF05900E15E0FE20
:10276300EFC39E501AEF2401FDE433FC900E115188
:10277300E41242F68F827583001201A40F80DC906D
:102783000E1151E4900E15E0FFF582758300E4020B
:1027930001A4900E97EBB1DE900E9751E4F1E21293
:1027A30056C212014C540F7C002FFFEC35F012552A
:1027B30076C98FF0120284900E9751E4F1E8125615
:1027C300C2F1DC540F2FFFEC35F0FE900E9A51E46A
:1027D300900002EE8FF00202A390000202016590C6
:1027E3000001020165900003020165E5F08FF0022C
:1027F300028412014C543FFDEF4DFF22D2241214E8
:10280300CED1827F801213F5D1827FA00214CC90A7
:102813000E78EB1225DEA3EDF030820F1254F22076
:102823001D0281A17A0C795D021FF5900B4CE044E7
:1028330004F0E4900E7BF0301D0241237BFF7A0C01
:102843007970121E25D21D301C0241171227FF1268
:10285300001A1217D4123F40F1F3121FA4740CF0A4
:10286300A37480F0900BD1E024E8FEE434FF900ED3
:10287300A7F0A3CEF0900F22E0900EA9D1CD900F38
:1028830023E07F4430E1027F50900EAB1222D1123D
:102893001E257D1A7F01D1EE7D1A7F02F124F0F10E
:1028A30035E4900B04F0900B06F0900B05F0900EBE
:1028B300A0120490000400007A0E797D91FB740E3F
:1028C300F0A3747DF07401123848900EA0120490A6
:1028D300000400017A0E797C91FB740EF0747C1273
:1028E300560FC3900E7DE094A0900E7CE0940F50A1
:1028F30024121FA4740CF0A37490F0900E7CE0FEDD
:10290300A3E0FF900B34EEF0A3EFF0900EA7EE12CE
:1029130022CF121E25900EA01204900005100091E4
:10292300FB740EF0747E12560F900E7EE030E009B9
:102933007BFF7A0C7997121E25900E7EE020E10929
:102943007BFF7A0C799B121E25900E7EE020E20914
:102953007BFF7A0C799F121E25900E7EE020E309FF
:102963007BFF7A0C79A3121E25900B52E030E0090D
:102973007BFF7A0C79A7121E25900B52E030E009F9
:102983007BFF7A0C79AB121E25900B52E030E009E5
:102993007BFF7A0C79AF121E25900B52E030E509CC
:1029A3007BFF7A0C79B3121E25900C4AE0606EE42B
:1029B300F0900EA01204900006000091FB740EF03C
:1029C300747D123844E4900E7CF0900E7CE0FD257B
:1029D300E0247DF582E4340EF583E0FF74382DF5B1
:1029E30082E4340BF583EFF0900E7CE004F0E0B466
:1029F30005D8E4900B3DF07B017A0B7938900E9665
:102A0300F0A37406F07F807E0112174C7BFF7A0CD3
:102A130079B780067BFF7A0C79BB121E25121E172D
:102A2300301C0281A1900B05E030E00281A1F1F39B
:102A3300900F23E0900B4C30E006E04408F0800454
:102A4300E054F7F0900F20E0FFA3E0900B4ECFF09F
:102A5300A3EFF0900F25E0900B4DF0900F24E09042
:102A63000B51F0E0FF900B06E06F70026110E490F1
:102A73000E7CF0900B51E0900B06F0900B52E0307F
:102A8300E012900B4D91E81223042401121FAE9023
:102A93000BE1D1BA900B52E030E21A900B4DE0FDFE
:102AA300E4FF1214E7900BE51223042401121FAE76
:102AB300900BE5D1BA900B52E030E31D7DAC7F0162
:102AC3001214E71214D71214D7900BE9122304241B
:102AD30001121FAE900BE9D1BA301E0B300D0890D6
:102AE3000B4DE0FF124964900E7CE06020121FA49E
:102AF300740CF0A374C4F0900B4DD1C9783C12044C
:102B030011900EA912046B1222D3121E25E4900B0E
:102B130005F0900F17E0900B53F0E0700281A19045
:102B23000B04E0FF54F0FE900B53E054F06E603E54
:102B3300EF540F12567754F04F900B04F0E054F01B
:102B4300C4540FFF900E7CF07843E654E3F6EFD3C2
:102B5300940C4006E64410F68014900E7CE0D39467
:102B6300057843E640054408F680034404F6900BD9
:102B730004E0FF540FFE900B53E0540F6E7002817C
:102B8300A1EF54F0125677540F4F900B04F1EB1250
:102B93003053900B52E0C330E501D340691214095E
:102BA300900B52E020E4028175E0C330E001D34092
:102BB3000E91D0122304121FAC900BE112046B9000
:102BC3000B52E0C330E201D340151255BD121593E9
:102BD300900BE5122304121FAC900BE512046B90CB
:102BE3000B52E0C330E301D350028175900E7C7425
:102BF300ABF07A0E797C12154A900BE9122304127A
:102C03001FACF1E5806C900E947401F0A3740BF08B
:102C1300A37400F1EB1223EDEF604B7843E644011C
:102C2300F6900C4B7401121FA3740CF0A374D8F02C
:102C3300900B001241ABF0900B02E0FFA3E0900E6B
:102C4300A9CF1222CF121E251256A71241C7EF6039
:102C53000D1256A7A3E0FCA3E0FDB10380147BFF94
:102C63007A0C79F080091254F97BFF7A0C79FD1202
:102C73001E25121FA4740DF0A37404F0900B54D1FD
:102C8300C9900B55125582F0900B5612559CF0903B
:102C93000B57E0FF900EADE41222CF121E2522C285
:102CA300AC900DF3E0C394CE4006D2ACD1D4D32282
:102CB300900DF1E0241DF582E4340DF583EFF090DF
:102CC3000DF11232D904F0D2ACD1D4C322900B54FB
:102CD300E0FF91A2900B55E0FF91A2900B56E0FF0D
:102CE30091A2900B57E0FF91A2900BE122FF900E6F
:102CF300A012046B7A0B7968900EA47401F0A322DE
:102D0300900E91EEF0A3EFF0A3ECF0ED124220EC65
:102D13005407AF05A3F0A3EFF0900B52E030E15F4F
:102D2300900E92E0543F44C0900E95F01242077803
:102D330006CEC313CE13D8F9547FFF900E94E0FE52
:102D4300C433333354804F900E96F0900E93E0FCCF
:102D5300A3E0FDECC313ED13900E97F0ECC31354F3
:102D630003A3F07B017A0E79951242A8900E99EF96
:102D7300F0900E98E0FEEF54FCFFEE4FF0C1089088
:102D83000E91E0FCA3E0FDD39463EC9400404BE090
:102D9300543F4440900E95F0EDAE047806CEC31335
:102DA300CE13D8F9543F4440900E96F0ECC454012E
:102DB300FF900E94E025E0543E4F44C0900E97F0F0
:102DC300900E93E0FEA3E07805CEC313CE13D8F99B
:102DD300543F44C0900E98F0802B900E91E0FAA3DC
:102DE300E0FBFFD179900E95D171D1B2900E93E0B3
:102DF300FAA3E0FB7C007D0AFFAE021201D8900E1D
:102E030097D171D1B2900BE012140C900B52E030B9
:102E1300E459E0C330E001D3400E91D012230412F1
:102E23001FAC900BE112046B900B52E0C330E20134
:102E3300D340151255BD121593900BE512230412BE
:102E43001FAC900BE512046B900B52E0C330E3010F
:102E5300D34018900E9974ABF07A0E799912154AF3
:102E6300900BE9122304121FACF1E57F0122EF540A
:102E73000F4403F0AF037C007D0AAE020201D85376
:102E830090FB439004222024037FFF221214CED10F
:102E930082EFB401047FC080027FC21213F5D18296
:102EA300120026EF541FFFC3741F9FFF0214CEEDC1
:102EB300540F4403A3F02212046B900E7C7401F0B0
:102EC30022A3F0900E8CE0900EA7FFE4F0A3EFF0A6
:102ED30022900DF4E030E0121232B0400D201F0AB0
:102EE300C2AC1232C612319CD2AC22900E91EDF0DC
:102EF300AD073024271214CE900E91E0541FFEC369
:102F0300741F9E541FF0D182EDB40103E08006903C
:102F13000E91E04440FF1213F51214CE22E0FD7F20
:102F230001D1EE7F01D189900BD3EF22E0FD7F0227
:102F3300D1EE7F02D189900BD4EFF022900EA01234
:102F43000490000000007A0B794A91FB1256EA7450
:102F530040F1DE900EA01204900000008091FB74FB
:102F63000BF074D1F1DA900EA0120490000001006E
:102F730091FB740BF074E1F1DA900B52E0F4702CD6
:102F83007B017A0B794A900E99F0A37440F0E4FF29
:102F9300FE1220111237E41241C01256DA12201128
:102FA3001237EB1241C07410F012200D900B52E057
:102FB300B4FF02E4F012554EE04440F0900B4CE0B5
:102FC30054FEF0E4900B58F0900B64F0A3F0900BD8
:102FD30067F0900B53F022A3F07410A3F07F02026A
:102FE300384C900BE902046BF07B017A0B79542285
:102FF30020823B1214CEC2950000000000000000A6
:103003000000E4900E91F0900E91E0FFC3940850FD
:103013001B7E00113A900E91E025E02416F582E420
:10302300340F1132900E91E004F080DBD29522F53B
:1030330083EEF0A3EFF022AD07AC06ECFF121725E9
:10304300AE07AF05121725AD07EEFEEDEEEDFF223D
:10305300900E911217ED900F19117DEF12019290BE
:103063000F1B117DEF120192900F1D117DEF1201C5
:1030730092900F1F117DEF020192E0FF900E91E0FD
:10308300FBA3E475F001120243A9F0FA22C0E0C0E9
:10309300F0C083C082C0D075D008309833C29890F6
:1030A3000DF2E0FFC394CE4017900DF5E599F0EFD4
:1030B30094D050083105747E11F404F0D220802698
:1030C3003105E59911F404F0E0C394C84002D2201D
:1030D300309913C299301F02800A51B0400651C67D
:1030E300319C800231A4D0D0D082D083D0F0D0E004
:1030F30032F0900DEFE075F0D084E5F0F0900DF232
:10310300E022900DEFE0FF04F0744C2FF582E434DD
:103113000CF58322900DF2E070037FFF22C2AC9086
:103123000DEEE0244C310FE0FF900DEEE004F011C2
:10313300F814F0C220D2AC22E4FF31926016E060B2
:10314300135418FFBF080D318B900E7C747FF0E48D
:10315300FF1216A27F0131926017E0FF601354182B
:10316300FFBF080D318B900E7C747FF07F01121628
:10317300A251B850123117318B7D801238A8318B90
:103183007D8012281280EA227B017A0D79F82212BF
:103193001737900DF7EFF0F42214F0A3E054FEF08C
:1031A30022900DF4E04401F022C28EC2AB75981058
:1031B300D29C7F007EC27D017C0031EE538EF07580
:1031C3008BFF53890F43892031A454FBF0C220E4C1
:1031D300900DEEF0A3F0A3F0A3F0A3F0A3F0C29937
:1031E300C298D2ACD2BCD299D28E22900E8B12044A
:1031F3006B51A1120514328400000960327F000074
:1032030012C0327700002580327200003840326DE0
:1032130000004B00326000007080325B00009600BB
:1032230032560000E10032490001C200324400037B
:103233008400323F0007080000003291758DCC8076
:1032430008758D988003758D30E58E54F44408F528
:103253008E804B758D988008758D648003758D30D5
:10326300E58E54F44401F58E8034758D988008758D
:103273008D758003758D30538EF48022758D988003
:1032830003758D30E58E54F44402F58E8010758DF0
:1032930030538EF4900E8B12049000002580900E14
:1032A3008BE0FCA3E0FDA3E0FEA3E0FF22900DF37F
:1032B300E0D3940022900DF2E0D394004003D38036
:1032C30001C322900DF0E0241DF582E4340DF58353
:1032D300E0F599900DF0E004F0E075F0D084E5F0AE
:1032E300F0900DF3E022EF24F7604024F7603624DA
:1032F300ED603E24ED602824ED601E24DB60142481
:10330300DA600A24B5702A7F007EE180287F007E80
:103313009680227F807E70801C7F007E4B80167F8C
:10332300407E3880107FC07E12800A7F607E0980D5
:10333300047F807E257D007C0031EEEEFF2253D991
:10334300BF759003B11253903B43A03DD295914773
:1033530091C943800491F291D931AC1212DB121658
:10336300731215F6900BCEE06004A3E07003121500
:10337300F67B017A0B7938900E99E4F0A37405F08B
:103383007F807E01122011E4900C4AF0900B38E00C
:10339300D3648094FF40187B017A0B7938900E999F
:1033A300E4F0A37405F012200D900C4A7401F09020
:1033B3000DF67402F0900DF6E0FFC39407503974D4
:1033C300362FF582E4340BF583E0FFD3648094FF5A
:1033D3005008C3EF648094A05016900C4A7401F017
:1033E3007E007F057D30FB7A0B79381206FE80085C
:1033F300900DF6E004F080BDE4900B3DF0A3F0C225
:1034030000900DF67402F0900DF6E0FFC3940750A0
:103413001B74362FF582E4340BF583E064306004CB
:10342300D2008008900DF6E004F080DB30000A90B3
:103433000B38E06004A3E07006900C4A7401F0B10D
:103443003A02188D43B203E4F5B943B9809163435B
:10345300B9C09163E5B930E5FB75A90343B6902282
:10346300E4FFFE0FBF00010EBE01F8BFF4F522D248
:10347300A7E4900E8BF0A3F09163900E8CE004F020
:103483007006900E8BE004F0C3900E8CE09458907D
:103493000E8BE06480948240DFC2A7E4900E8BF031
:1034A300A3F09163900E8CE004F07006900E8BE015
:1034B30004F0C3900E8CE094B0900E8BE064809483
:1034C3008440DFD2A72275A2F075A140E4F5F8D2BB
:1034D300F9D2F8C2FF22E47841F608F675D10775F0
:1034E300BB1E75BA1F75BCFC75E8C243E60822789B
:1034F3003C12047700000000E4F5C8538E0F75CB2F
:10350300F075CA5C74FFF5CDF5CCD2ADD2CA227585
:10351300D6FF75D5FF75D48C75F3FD75F2FF75F184
:10352300FF43A4C153A4F375A5C775A6FD75E103B5
:10353300E4F5E243E24022E59620E7FB7596017548
:103543009708E59620E7FB759607759707E596209C
:10355300E7FB759609759707E59620E7FB75960BCC
:1035630075970775D7E0E59620E7FB75960F759776
:103573008043E602D2AFE59620E7FB759601759787
:1035830001227BFF121E25E5C930E63A783C12047E
:1035930011EF2432FFE43EFEE43DFDE43CFC900EDB
:1035A3009F12046BB1CA401E783C120411900E9F07
:1035B300E0F8A3E0F9A3E0FAA3E0FBD31203ED40A4
:1035C30005121FBE80DE22D3E51D9400E51C940086
:1035D30022B1CA4034ED60317401251FF5827400B5
:1035E300351EF583E0120192051FE51F7002051ECB
:1035F300E51D151D7002151CD11A1DC3E51E940689
:1036030040CFE4F51EF51F80C8C3E51C94064003B4
:10361300D38001C3922622740129F9E43AFA229055
:103623000EA8ECF0A3EDF0C3E51C9406505EC3E5D1
:103633001C9406504A900EA8E07002A3E06040126A
:10364300014CFF7401251BF5827400351AF583EFD5
:10365300F0051BE51B7002051A051DE51D7002052B
:103663001CD11A900EA9E024FFF0900EA8E034FFBD
:10367300F0C3E51A940640B6E4F51AF51B80AFC310
:10368300E51C94064003D38001C3922622900EA129
:10369300EFF07B017A0E79A17D017C008081900E91
:1036A30098EFF01217F600000000007F051213F5E3
:1036B3000000000000120026900E98EFF053903B9C
:1036C30043A03DD295E0FF22900E8EEFF0900E9630
:1036D300E0A3F0900E96E0FF14F0EF6057900E8E8B
:1036E300E0FF1217F600000000007F061213F590AA
:1036F3000E8EE0FF1217F60000000000A312042A4A
:10370300900EAA12046B7F0212382C0000000000F6
:10371300900E93E0FBA3E475F001120243A9F0FAC3
:1037230012014CFF1213F5900E8EE0FFD1A1EF2092
:10373300E0F5809F53903B43A03DD295900E97E0D8
:10374300FF227A0B794AF1BE7440F0E4FFFE1217B0
:103753004CF1E4F1C01256DA12174CF1EBF1C074DC
:1037630010F07F007E0112174C900E93120490000C
:103773000000007F0212183F900E8F120490000089
:1037830000007A0B794AF1DC1256EA7440F1C71251
:10379300049000000080F1DC740BF0A374D1F0748A
:1037A30010F1C712049000000100F1DC740BF0A3C8
:1037B30074E1F0A37410F07F02C1CB7B01900E96ED
:1037C300E4F0A322A3F07F02D1CB900E8F22FF90CF
:1037D3000E8F12046B7A0B799C900E937401F0A3F5
:1037E300227B017A0B79D1227B017A0B79E122903A
:1037F3000EAE12046B900EAEE0FCA3E0FDA3E0FE60
:10380300A3E0FF78101203FE1213F5900EAEE0FC56
:10381300A3E0FDA3E0FEA3E0FF78081203FE12136A
:10382300F5900EB1E0FF0213F51213F5900EAAE026
:10383300FCA3E0FDA3E0FEA3E0FF80B3740BF074F0
:10384300F2A3F07414A3F07F031217F60000000034
:1038530000900EA0E0FCA3E0FDA3E0FEA3E0FF9038
:103863000EAA12046B7F03112C900EA7E0A3F09015
:103873000EA7E0FF14F0EF601E000000000012002E
:1038830026900EA4E0FBA3E475F001120243A9F015
:10389300FAEF12019280D853903B43A03DD295900A
:1038A3000EA8E0FF22900E78EB1225DEE4FD900BCC
:1038B3008CE0FF900B58E06F700241A4900B8BE0FB
:1038C30024DB700221D424F570024193242FB41811
:1038D30000400241A19038DF12565E730239320272
:1038E3003AA102394A0239530239B80239BD0239C1
:1038F300FF02395B02396D02393E0239B0023AA147
:1039030002397F023992023AA1023A3C0239270274
:1039130039440239C6023A24023A8B0239EF023A99
:1039230065023A78E4900B67F0900B65F041A1D102
:10393300CF7F01D1F9D1CF7F028076D1CF7F0780AE
:1039430070D1CF7F09806A900B9C122F20F021EA5F
:10395300900B9C122F2F21EAF1D47F05D1F9900B04
:10396300D7E0FCA3E0FD7F068047900BD5E0FCA3E6
:10397300E0FD7F05D1F9F1D47F068035900B9CE003
:10398300FF1232E9900BDFEFF0E0FD7F0180199029
:103993000B9C12140C900B9C12140C900BE0EFF088
:1039A300900BD2F0E0FD7F02121EEF803AF1D47F3C
:1039B30008D1F9803212347241A112554E7B107D29
:1039C30010800712554E7B307D307F0112178A41DC
:1039D300A1900B52E054D2F0E0FF900B9CE0542DE9
:1039E300FEEF4E900B52F012374541A1900F22E0AB
:1039F300900B68F0900B667401F041A11255DB90B7
:103A03000B8B7411F0123745E4900E7BF012346384
:103A1300900E7BE004F0E0C3946440F143EF9080A8
:103A23007D900B9CE06009D21C43A404C282806E8B
:103A3300C21CD28253A4FB8065900B9512570A9047
:103A43000E9EF07F01121593900BE9122475FB90E3
:103A53000B95E0FFE4FCFDFEEB125653FC122FE541
:103A6300803C900B4CE054DFF07A0B79D112555621
:103A73004410F08029900B4CE054EFF07A0B79E17D
:103A83001255564420F08016900BD0E004F0800EBF
:103A93001222E17F007E107D007C0012230F12555D
:103AA300DB900B9AE0FF900B67E06F700261B0E46C
:103AB300FFFE7D10900B96122474FBC31203ED409E
:103AC3003330820F900B67E064FE700261B01256D0
:103AD3000361B01222EDC3900E7B125505900E7B4D
:103AE3001223061256D21222FB122CF01255AEF0FC
:103AF3007F03619E7FFF7EFF7D0F7C00900B9612FC
:103B03002475FBC31203ED7028900D8393F91256AD
:103B13001C93900E8EC91225DE900B9BE0FF900E36
:103B230091E4F0A3EFF07B017A0B796812113080F6
:103B33006CE4FFFE7D0FFC900B96122475FBC31201
:103B430003ED401A1222EDF1957B017A0B7968900F
:103B53000B9BE0FD1241C0EDF0122011803FE4FF0A
:103B6300FE7D0EFC900B96122475FBC31203ED40F1
:103B7300361222EDC3900E7B1254E0900E7BD1C718
:103B8300E4FDFC1222FB2400FFEE3410121FB112DD
:103B930022FB122CF01255AEF07F02114C900B9ABF
:103BA300E0900B67F08006900B6774FDF0900B8D2F
:103BB300E0FF900B65E06F7002C192E47D10122468
:103BC3006FFBC31203ED5002A10730820F900B6508
:103BD300E064FE7002C192125603C192900B9012E0
:103BE3002304FFF1DD122304C3900E8712550590C1
:103BF3000E871223061256D2F1DDD1C7EE540FFE03
:103C0300EE4F7011900B07F0900E87122304D1C171
:103C13007F0312183FD1BA900E871223041256E283
:103C230012046BF1CBFE900E87122475D1AF1203F1
:103C33005B900E7F12046BD1BA900C06122304FF23
:103C430012035B900E8312046B900E7F122304FF0A
:103C5300900E7B122475FBC31203ED601BE4FF7E01
:103C630010FDFC900E7F122475FB1202D0900E8380
:103C730012046B900E83801B900E83122304240185
:103C8300121FAE900E7B122475FBC31203ED700E50
:103C9300900E87122304FFD1C17F0312183F900EA9
:103CA30087122304FF900C06F1E01223041237D18C
:103CB30012558C7F031255274008121E17E4900BF0
:103CC30007F0900E87122304F1E7900E7812247800
:103CD300900EA4C91225DE1256957F03D1E112225C
:103CE300E11206DAEF7002C175121FA4740DF0A37E
:103CF3007446F0900E871223041242001222D3124C
:103D03001E25C175E47D0F12246FFBC31203ED4022
:103D13003C900B901222F0F195900B9412570AFDF0
:103D23001237C0EDF012174CF1C21222E1900B943E
:103D3300E0FD1241C0EDF0122011D1E31222E11295
:103D430006DAEF6006900D8C121E1AC175E4FFFEB1
:103D53007D0E122471FBC31203ED5002C17F900B41
:103D630090122304FFD1D7122304C3900E8112545F
:103D7300E0900E81D1C7E4FDFCD1D71223042400C7
:103D8300FFEE3410121FB1D1D7D1C7EE540FFEEEA0
:103D93004F7011900B07F0900E81122304D1C17F55
:103DA3000212183FD1BA900E811223041256E2EE8A
:103DB300F0A3EFF0F1CBFE900E81122475D1AF1278
:103DC300035B900E7DEEF0A3EFF0D1BA900BCA1215
:103DD3002304FF12035B900E7FEEF0A3EFF0F1C21A
:103DE300900E7BE06E7003A3E06F600FF1CBFE904B
:103DF3000E81122475125653FC8021900E80E0240C
:103E030001FF900E7FE03400FE900E7BE0B50613B9
:103E1300A3E0B5070E900E81122304FFD1C17F02E8
:103E230012183F900E81122304FF900BCAD1DA12AD
:103E330023041237D112558C7F02125527400812E2
:103E43001E17E4900B07F0900E81122304F1E79004
:103E53000E78122478900EA4C91225DE1256957F8F
:103E630002D1E11222E11206DAEF6006900D8C1204
:103E73001E1A900B8DE0900B65F08013E4FFFE7D1E
:103E83000D122471FBC31203ED900B6574FDF0E575
:103E9300C930E60FD21E124821A20B50028001C383
:103EA300921B22301E05C21E12004E222FFFEE3A35
:103EB300FEED39FDEC38FCE4FB7A10F9F822900EA4
:103EC3009302046BA3A3E0FEA3E0FF22900B9CE00C
:103ED300FD7C0022900E8112046B900E8122114C06
:103EE300900B94E0FF7E00789C7C0B7D0122900E6A
:103EF3000DE0FCA3E0FD900E8BEFF0A3ECF0A3ED3F
:103F0300F012422D900E8CE0FEA3E0FF900E8BE0AA
:103F130025E024F2F582E4340BF583EEF0A3EFF011
:103F2300900E8F120490000500001237DC740BF022
:103F3300A374F2F0A37414F07F031236CB900EA097
:103F430012049000050000122CFB113F900BF5E0CA
:103F5300900BD1F0900BFCE0FFA3E0900BD5CFF0DA
:103F6300A3EFF0900BFEE0FFA3E0900BD7CFF0A3FD
:103F7300EFF0900C01E0900B4AF0900C02E0FFA3ED
:103F8300E0900BD9CFF0A3EFF0900C05E0900B4B32
:103F9300F022C39400FFEE9400FEED940FFDEC9429
:103FA30000FC900E7B12046B900E7BA3A3E0FEA398
:103FB300E0FFEE541FFEE4FDFC900E7B12046B90B9
:103FC3000E7DE0FEA3E0FF22900B94E0FFE4FCFDF6
:103FD30022900B9CE0FCA3E0FD22900E8712046B61
:103FE300900E8722FF900EA002046BE49009F4F078
:103FF300A3F090060EF0A3F09009F2F0A3F0900660
:104003000CF0A3F0784DF608F6784BF608F6C20EDE
:10401300D20DC212C211C210C20F22900E9DECF03B
:10402300A3EDF01213F5900E9DE0FF1213F5900E21
:104033009EE0FF0213F5C2A832C0E0C0F0C083C007
:1040430082C0D075D000C000C001C002C004C0054A
:10405300C006C007783C120411E4FAF9F8EF240112
:10406300FFEA3EFEE93DFDE83CFC783C12045FC2FA
:10407300CFD007D006D005D004D002D001D000D0D5
:10408300D0D082D083D0F0D0E032C0E0C0D075D0A1
:1040930000C000C001C005C006E5BBB41E1CE5BEE0
:1040A300FEE5BDFDEEED7806CEC313CE13D8F97948
:1040B30032F7EE19F775BB09801AE5BEFEE5BDFDC3
:1040C300EEED7806CEC313CE13D8F97942F7EE1985
:1040D300F775BB1EC2EDD006D005D001D000D0D0FD
:1040E300D0E032E0FEA3E0FF900E11EEF0A3EFF07C
:1040F300900E11E0FEA3E07803CEC313CE13D8F9DC
:104103007A0E791331B704F0122011121FA4740D23
:10411300F0A37453F0900E1131ABF07B017A0B795D
:10412300081207BD7B017A0B7908900E13E0FFE4B8
:10413300FCFDFE5117900E15EB1225DE900E14EFC9
:10414300F0BF0107900B8AE020E047900B1374AA9D
:10415300F0A33196900E9E7402F0121593900E15F3
:104163001222E431A3F0900E14E0FFA31222E41212
:104173001593121FA4740DF0A3745CF0900E181223
:1041830023045100319C1207BD319C31A331961297
:10419300159322F0900E14E0FF7B017A0B79132222
:1041A300120003900E9EEF22E0FFA3E0CF900EA734
:1041B300F0A3EF222400FFEE3402FE7B01900E9960
:1041C300E4F0A322900E91EEF0EF51205107780313
:1041D300CEC313CE13D8F97A0E799331B704F01204
:1041E3002011900E92E0510F088002C333D8FCFFD8
:1041F300900E93E05F6F7F0160027F0022FF900EBD
:10420300A702046B900E91E0FEA3E0225407FF7413
:1042130001A80722900E1812046B7F0122A3F0EE6F
:10422300541F900E91F0A3EFF022900EA012049071
:1042330000050000122CFB12383F7F007E007D0535
:104243007C00021823900DF7EB1225DEA3EDF0E4BA
:10425300FF1217378F25E525B4FF087BFF7A0D7909
:10426300628036E5256035E52554186408702D9085
:104273000DF71222E451A0E4FF1216A2900B33EFC4
:10428300F0900DF71222E4900B3312278AEFD394A8
:10429300004009900DF71222E4121E2522A3E01418
:1042A300900E7CF022EB1225DBE4A3F0FDFC900ED4
:1042B3009A1222E451F6F9E4FBFA900E9DE0C3133F
:1042C300F0E930E004E04480F0E9C313F9900E9D77
:1042D300E030E103649AF00BBB00010AEB64084A87
:1042E30070D80DBD00010CED64044C70C1900E9D9F
:1042F300E0FF228D828C8302016512014C54C0FFC2
:10430300BFC00951A8EF7004FE7F0122E4FEFF2223
:1043130012014C54C0644070201227E254C0644020
:1043230070171227DC54C0FFBFC00E1227E854C019
:10433300FFBFC0057E007F0122E4FEFF2212014C75
:104343005470643070201227E25470643070171276
:1043530027DC5470FFBF300E1227E85470FFBF30C4
:10436300057E007F0122E4FEFF227E447D07AC0729
:104373000FA804E6AB060EA803F6DDF2123FEED259
:1043830010D3227F51718E7F5180DFA807E6900EF4
:10439300D5F0E804F8E6900ED4F0EF2402F8E690A6
:1043A3000ED3F0EF2403F8E6900ED2F0A807F6A39D
:1043B300E0FEE80471C3240271C32403F8A60622B5
:1043C300F8A606A3E0FEEF22F1897057900F01E0F3
:1043D3007002A3E0704D900F05E07004A3E0640742
:1043E3007041900ED07451F0A37444F0900ECF74CA
:1043F30007F0900ED1E0FF04F0A807E6FF900ED07F
:10440300E0FE04F0A806A607900ECFE014F0E070DB
:10441300E17F51718EF194900F0E74029133740702
:10442300F0D21922900F09E4F0A37400F07451A3A1
:10443300F0900F07E4F0A322900EFFE06480600287
:10444300A187900F01E024FE602E146050240260C7
:1044530002A1DF900F02E06002A1DFA3E07002A3DC
:10446300E06002A1DF900F0974FFF0A37411F0A3C1
:1044730074CE91337412A1DC900F02E06002A1DFCD
:10448300A3E07002A3E06002A1DF900F0974FFF0C4
:10449300A37411F0A374FC9133746BA1DC900F022D
:1044A300E0FFC394044002A1DFEF64036002A15C58
:1044B300900B36E0FF947F5008C3EF648094A050C4
:1044C300409012D9B1F4900ED174FF1225DE9012F0
:1044D300D9740193F5828E83E4930425E0B1FED170
:1044E30008506B900ED11222E48E82758300120164
:1044F30065FF74D62EF582E4340EF583EFB1EC80BC
:10450300DE7B017A0B7936120003EF04B1FED1088A
:104513005031EEC39411502B74362EF582E4340BD4
:10452300F583E0FDEE25E024D8F582E4340EF5832F
:10453300EDF0EE25E024D9F582E4340EF583E4B101
:10454300EC80CBEF25E0900ED6F0A37403F0D18975
:10455300740EF0A374D6F0801C900F02E075F00285
:10456300A424D3F582E5F03412F583B1F4900F0956
:1045730074FF1225DE900F091222E412014CFF9101
:1045830034EF8055900EFFE064817050900F03E08C
:104593007004A3E064027044900F01E024DE601C09
:1045A300047039900F02E07033900F0974FFF0A389
:1045B3007412F0A3745091337409801D900F02E0BC
:1045C300701A900F0974FFF0A37411F0A374E0F054
:1045D3009011FBE493FF9134EFF0D219301909D114
:1045E300914005EEF0A3EFF022F0900ECFE004F03F
:1045F30022E493FE740193AA06F922900ED0F0E40C
:10460300900ECFF022900ED0E0FF900ECFE0FEC3CD
:104613009F22F1897026900F02E07020900F01E035
:1046230024FD601124027014D189740BF0744A9133
:10463300327440800491277407F0D219301909D1DC
:10464300914005EEF0A3EFF022900EFFE06421709D
:1046530026900F02E07020900F01E024FD6011040A
:104663007015D189740BF0A3748A9133744080045C
:1046730091277407F0D21930190B7403D1934005B5
:10468300EEF0A3EFF022900F097401F0A32274025D
:10469300900F0EF0900F05E0FEA3E0FFD3900F08FC
:1046A300E09F900F07E09E22900F03E07002A3E0CB
:1046B3007027900F00E014601324E160111460115F
:1046C30014601014601024237042E1C1E1A2024F70
:1046D300DD61CB025017024802900F03E07004A380
:1046E300E064027027900F00E024FE601314601250
:1046F30024FA601014600F14600F240A700EC115A1
:10470300800B8040C14C02503512506422900EFF42
:10471300E0B4A123900F01E0701D900F05E0700439
:10472300A3E064017011900F02E014700A784FE661
:104733007851F6F194D219301909900F0E74029141
:104743003304F022F189703D900F01E07002A3E081
:104753007033900F05E07004A3E064017027900F9D
:104763000974FF20210BF0A37400F0A37418F080E8
:1047730009F0A37400F0A37419F0913404F0900FBE
:104783000E04F0D21922900EFFE064A122900F0EC6
:10479300F0900F09E4F0A37400F0A37451F0229099
:1047A3000EFFE0B4A117900F01E07002A3E0700DBB
:1047B3007402F190E4900F07F0A3F0D21922900E47
:1047C300FFE0B42123900F01E07002A3E0701912FF
:1047D3005309D39407EE9400500E7403F190900F95
:1047E30007EEF0A3EFF0D21922EFC330E001D3922A
:1047F3000BEFC330E101D3920C220FBF00002290D4
:104803000EFFE0B42117900F05E07002A3E0700DD6
:10481300900F01E0FEA3E0FF1247FDD21922511AC7
:10482300900F0CE060022127201302212753E6FD9D
:10483300E59620E7FB7148E59620E7FB759696E53C
:104843009620E7FB900607E597F0C374F0784E9641
:10485300FF74011896FEE0FD7C00C3EF9DEE9C50B3
:10486300022112C21390060EE0FEA3E0FF90060A97
:104873009157C3ED9FEC9E500D900607E0A3F0E423
:10488300A3F0C201801590060BE0FF900608F0909C
:104893000607E0C39F900609F0D201900608E09056
:1048A300060E913E2401F58274083EAB82FA7F2204
:1048B3003128900609E0600BFD7C007A087B017FBC
:1048C300223128E59620E7FB759614E4F59730012D
:1048D3000F900609E0FF90060EE4F0A3EFF08012BC
:1048E300900607E0FF90060FE02FF090060EE034ED
:1048F30000F0900607E0784E26F618E436F6D30863
:10490300E6940018E694004003D38001C3920EC3DB
:10491300784EE694EF18E694014003D38001C392E6
:104923001243E60222914E6037ED1D70011C144CB8
:10493300700CE94480F596E59620E7FB801FE94477
:10494300C0F596E59620E7FBE597F0A3ED1D700112
:104953001C144C70EEE59620E7FBE4F596E597F022
:1049630022900E91EFF0200D021121300D52900E86
:1049730091E0FF90060CE475F001120243FC741001
:1049830025F0F58274063CF583EFF0C390060DE045
:1049930094F090060CE094014004E4F0A3F0784C0A
:1049A30006E6187001069146C394EFEE9401500297
:1049B3008001C3920DC3EF9440EE94004002112195
:1049C30022900F0DE06401604D30144AC214E59645
:1049D30020E7FB9137E4900EFEF0E59620E7FB75A8
:1049E3009696E59620E7FB900EFEE597F0E064408F
:1049F300600DE59620E7FB759616759710800C7A87
:104A03000B7B8A7D407C007F233128E59620E7FBE2
:104A1300759614E4F59722900F11E0600261265316
:104A2300E6FDE59620E7FB7148E59620E7FB7596E2
:104A330091E59620E7FB900E92E597F0E030E002D7
:104A4300612391464E70026123C217D3EF9440EE67
:104A5300940040089006027440F08007784CE6907A
:104A63000602F09009F2E0FEA3E0FFC39006059171
:104A730057900602E0FDC39FE49E500AA3EDF0E4C5
:104A8300A3F0C2018015900606E0FF900603F090A4
:104A93000602E0C39F900604F0D201900603E09063
:104AA30009F2913E2410F58274063EAB82FA7F220E
:104AB3007127900604E0600BFD7C007A067B107F73
:104AC300227127E59620E7FB759611759701300152
:104AD3000F900604E0FF9009F2E4F0A3EFF08012D8
:104AE300900602E0FF9009F3E02FF09009F2E03422
:104AF30000F0900602E0FFFDC3784CE69DFD18E64A
:104B03009400FCF608EDF6C394EFEC940150028098
:104B130001C3920DEFC394404003D38001C3920FAE
:104B230043E60222914E601CE59620E7FBE9543FE1
:104B3300F596E59620E7FBE0F597A3ED1D70011CC4
:104B4300144C70EE2275960E75970222900EFFE0BC
:104B53006002811E900F03E07002A3E06002811ED9
:104B6300900F05E07002A3E06002811E900F02E047
:104B7300146016046002811E900F0F7403F0900FEF
:104B83000C74019126F0D21922900F0F7404F0E5F2
:104B93009620E7FB75960E759701E59620E7FB7562
:104BA3009612759720E59620E7FB911FE59620E77F
:104BB300FB7148E59620E7FB759612759784E59699
:104BC30020E7FB759615759780E59620E7FB7596AC
:104BD30013759740E59620E7FB911FE59620E7FBC9
:104BE3009137E59620E7FB759612759704E59620B5
:104BF300E7FB759613759740E59620E7FB911FE455
:104C0300900F0C9126F0D216D217D218C21AC213E3
:104C1300C214D222919012004ED2192275961075A9
:104C2300974022F0900F0DF0900F10F0900F11F0BD
:104C3300900F122275960E75970322FD7C00E0FEFD
:104C4300A3E022784BE6FE08E6FF22A9078B828ABF
:104C530083ED4C2274F09FFF74019EFEF0A3EFF0EE
:104C630022900F12E064016023301820C218E596E9
:104C730020E7FB91377A0B7B4A7D407C007F2371D1
:104C830027E59620E7FB75961175970122900F1083
:104C9300E0703D30223A301637C222C216E5962024
:104CA300E7FB75960E7597017A007B467D087F2199
:104CB300F1BF900F3AE0F597E59620E7FBE4F5970F
:104CC300E59620E7FBE59620E7FB759611759701BE
:104CD30022C0E0C0F0C083C082C0D075D000C00045
:104CE300C001C002C003C004C005C006C007E596EA
:104CF30020E7FB759686E59620E7FB900EC9E597BE
:104D0300F0E59620E7FB759682E59620E7FB900E8B
:104D1300CAE597F0E59620E7FB759684E59620E7CC
:104D2300FB900ECBE597F0900EC9E030E202B1B3F1
:104D3300900ECBE0FF30E202D213EF20E3033014F6
:104D430004D21431C4900ECAE0FF30E102D216EF50
:104D530030E202D217EF20E303301804D218916433
:104D6300900ECAE030E00312508F900EC9E030E39A
:104D7300049190B193D007D006D005D004D003D0CE
:104D830002D001D000D0D0D082D083D0F0D0E03296
:104D9300300F1C301719784CE618467012E5962030
:104DA300E7FB7148E59620E7FB759611759701229D
:104DB300E59620E7FB75960775970FE59620E7FBC9
:104DC30075960975970CE59620E7FB75960B759715
:104DD3000CE59620E7FB759601759701900F0F740C
:104DE30002B1FC900F0C04F0A3F0900F10F0A3F0AD
:104DF300A3F022900ECDE04408F0E4900F0EF022D1
:104E0300900F00E0B40C005041904E13F828287323
:104E1300024E37024E39024E4D024E3B024E4D02B8
:104E23004E3E024E41024E4D024E44024E47024E4A
:104E330049024E4B8073E1650253E8025438024441
:104E43003B02547E614F8025D14E22900EFFE0B489
:104E5300011A900F01E07002A3E07010F157500C9B
:104E6300900F05E07002A3E07002D21922D1A57061
:104E730030900EFFE064817028900F01E07002A370
:104E8300E0701EF157501A900F05E07004A3E06420
:104E930001700EF148900F0E740212443304F0D2E5
:104EA3001922900F0FE0640422900F01E07002A317
:104EB300E06002E139900F05E07004A3E064027042
:104EC30075900EFFE0247F601314601E2402706649
:104ED300900F03E07002A3E0705C8008D1A57056C8
:104EE300F1575052F148D219804CD1A57048900F18
:104EF30003E07042C20AA3E024FD6013248260141D
:104F03001460161460182481701E900F0C80129088
:104F13000F0D800D900F108008900F118003900FDC
:104F230012E024FF920AD219900F0974FF300A0489
:104F3300F1B58002F14D30190B900F0E740212443B
:104F4300337402F022900F0974FFF0A37400F0A3EE
:104F53007420F022C3900F04E09403900F03E094B5
:104F63000022D1A5704B900F05E07002A3E07041C1
:104F7300900EFFE024FE601D24027035900F01E0C7
:104F83007004A3E064017029900F03E07002A3E0B2
:104F9300701FD21922900F01E07002A3E0701290EB
:104FA3000F03E0700CA3E0FFE4FD1253125002D292
:104FB3001922F0A37400F0A3741EF0228B828A835B
:104FC300ED6016E59620E7FBEF543FF596E5962056
:104FD300E7FBE493F597A3DDF422900EFFE0B42101
:104FE30032900F01E07002A3E07028900F05E0708B
:104FF30004A3E06407701C900F0E7403F01244279F
:105003007407F0900F1374FFF0A37443F0A3748636
:10501300F0D21922900EFFE0B42116900F05E07034
:1050230002A3E0700C900F02E05403FF1247ECD28E
:105033001922900EFFE0B42127900F05E07002A320
:10504300E0701D900F02E014600D047013900F01C7
:10505300E0784FF6088006900F01E0784FF6D219FA
:1050630022900EFFE0B42123900F01E0701D900FFA
:1050730005E07002A3E07013900F02E014600804CF
:105083007009C221D21922D221D21922E59620E732
:10509300FB75960EE4F597E59620E7FB759691E58B
:1050A3009620E7FB519AFF30E210E59620E7FB7567
:1050B3009611E4F597900F0EF022EF30E410E59689
:1050C30020E7FB759611759780E4900F0EF0900F13
:1050D3000EE060022175900ECCE020E00221757B8A
:1050E300017A0E79FF7D087F2051CF900F02E09067
:1050F3000F0151A2F0900F04E0FE900F0351A3F0B3
:10510300900F06E0900F0551A2F0C219900F13E41F
:10511300F0A3F0A3F0900EFFE0546024E0600D24B0
:10512300E0600E2440700D124E0380081246AB80DF
:1051330003120022E59620E7FB75960EE4F59730FF
:10514300190DE59620E7FB7596117597408011E5DB
:105153009620E7FB759611759720900F0E7404F057
:105163007109A3E0B50608A3E0B50703D38001C323
:105173009215900F0EE064027076900ECCE020E161
:105183006FE59620E7FB759691E59620E7FB519A2C
:1051930020E45D20E05AA37402F0C3900F08E0946A
:1051A30040900F07E094004030900F091222E47DF5
:1051B300407F2051B6900F0AE475F04012022D9003
:1051C3000F08E024C0F0900F07E034FFF03015190A
:1051D300E07002A3E07012800D900F08E0FDA312AF
:1051E30022E47F2051B6124DF6E59620E7FB51AC41
:1051F300900F0EE0640360024199E59620E7FB758A
:105203009691E59620E7FB519A20E0024199A37419
:1052130040F0E59620E7FB759696E59620E7FB9030
:105223000ECEE597F0E0FD900F091222E47F2051A6
:10523300CF900ECEE0F9FF7E00900F0AEE8FF012B2
:10524300022D900F07E0FCA3E0FDD39FEC9E4010DE
:10525300E9FFED9FFFEC9E900F07F0A3EFF0802F87
:10526300E9FF900F07E0B4001AA3E0B50715900F0C
:10527300131222E4EA494B600A12054E5005124DFF
:10528300F6800C900ECD7420F0900F0E7404F0E5B0
:105293009620E7FB51AC22900ECCE597F0E022FE7E
:1052A300E0FDEDFFEEF0A3EF22759611900ECDE039
:1052B300F59722ED6015E59620E7FB8F9612014CDA
:1052C300F5977101E59620E7FBDDF222ED602EDD17
:1052D3000CEF4480F596E59620E7FB801BEF44C076
:1052E300F596E59620E7FBE5971201927101DDF251
:1052F300E59620E7FBE4F596E59712019222740107
:1053030029F9E43AFA22900F05E0FEA3E0FF22EF29
:1053130024FD60152482601814601C14602024810D
:105323007023900F0CEDF0801E900F0DEDF08017A1
:10533300900F10EDF08010900F11EDF08009900F99
:1053430012EDF08002C322E59620E7FB75960EEF7F
:10535300547FF597EF30E732ED7E5870027E48E5D3
:105363009620E7FB7596118E97E59620E7FB7596D9
:1053730091E59620E7FB71E020E3EE30E139E59615
:1053830020E7FB7596118E97802DED7EB070027E1F
:1053930090E59620E7FB7596148E97E59620E7FB3C
:1053A300759694E59620E7FB71E020E4EEE5962000
:1053B300E7FB7596148E97EFB48102D216EFB48291
:1053C30002D217EFB48302D217EFB40102C21AEF6D
:1053D300B40202C213EFB40302C214D322900ECF5D
:1053E300E597F0E022124EA5704A900F05E0700297
:1053F300A3E07040900EFFE024FE601D2402703491
:10540300900F01E07004A3E064017028900F03E0A3
:105413007002A3E0701ED21922900F01E07002A364
:10542300E07011900F03E0700BA3E0FF7D01711298
:105433005002D21922900EFFE0703F900F03E070EC
:1054430002A3E07035900F05E07002A3E0702B908B
:105453000F01E07025A3E020E7206016E59620E722
:10546300FBE4F596900F02E0F597900F0F7403F0AD
:105473008006900F0F7402F0D21922900EFFE064A1
:1054830080703B900F01E07002A3E07031900F0336
:10549300E07002A3E07027900F05E07004A3E064BE
:1054A30001701B900F0FE0FFB4040A900F0974FF03
:1054B300124FB5D219EFB40305124F48D219301960
:1054C3000A900F0E740212443304F0222400FFEEFC
:1054D3003402FE7B017A0E790FE4F0A3229400FFDD
:1054E300EE9400FEED940EFDEC9400FC02046B9030
:1054F3000B4CE054FBF07843E654FEF6E4900C4B7F
:10550300F0229400FFEE9400FEED9410FDEC940065
:10551300FC02046B7B017A0E798D1207BD7B017A45
:105523000E798D221236CB7BFF7A0D7944121E251C
:10553300900B07E004F0D3942822900002EE8FF042
:105543001202A3E92402F9E43AFA22900B52E0543E
:10555300EFF022787A7C0B7D017B017E007F1012B5
:105563000126900B4CE0227F407D007B011206FE5A
:105573007E0022F9900E9AE0FBA3E0FAA3E022E07A
:10558300FF900EA9E4F0A3EF22740BF0A3749CF038
:10559300900B94E0900E96F022E0FF900EABE4F0B7
:1055A300A3EF227BFFE0FFE4FCFD22740BF0A37466
:1055B30068F0900B9BE0900EA7227B017A0B795445
:1055C300900E9E7404F0E4FF22900E067401F0A383
:1055D300740BF0A3741FF022900B8CE0900B58F027
:1055E30022900E9AE0FF121498900E9BEFF022A3E4
:1055F300F0A37401F022EE8FF0120284900E9A222F
:1056030074FEF07BFF7A0D7922021E25A3F0A374AA
:1056130001F07F0302384C93FB740193FA74022266
:10562300900E09E0FEA3E022900E07E475F001223C
:10563300F582E4340BF58322900EA3E0FBA3E0FA9A
:10564300A3E0F92225E0242CF582E4340FF583222C
:105653002FFFEE3AFEED39FDEC382275F003A4C5B9
:105663008325F0C58322121E25900E8B221207BDBF
:10567300900E8F22FF900B04F0900B53E02274FFE7
:10568300F5F012024345F022E0FEA3E0FF900DF98E
:10569300E022900B94E0900EA7F022E4FD12275035
:1056A300900E0222900B00E0FEA3E0FF22E0FEA397
:1056B300E0FFE4FCFD22120026900DF7EFF02254E8
:1056C3000F75F00AA4FF227BFFE0FFE4FCFD22FF3D
:1056D300ED5407FDE4FC227410F07F807E0022FF6E
:1056E30012035B900E7B22740BF0A3744AF022FF2B
:1056F300EC4EFEED4FFF22900DFCE0FFA3E0229065
:105703000B52E04410F0227B017A0B799CE022904B
:105713000BD0E0D394002212041DD30203EDAF2B70
:0E5723001217378F2C22900E7DE0FFA3E0229C
:10F80000900F35EFF0900F36EDF0900F37EBF0756D
:10F81000E70075E60075A80053B2FCD291D290C201
:10F8200025007F0331990053903B43A03DD295754D
:10F830001400751500C3E51494F8504AAE14AF15C2
:10F840008E168F1775B7A575B7F1438F03AE16AF38
:10F85000178F828E83E4F0538FFC751100E511C37E
:10F8600094FF5013751200E512C394FF5005000574
:10F870001280F4051180E6B290E42515F5157402A6
:10F880003514F51480AF7F013199751000E510C370
:10F8900094FF5021751100E511C394FF50137512A8
:10F8A00000E512C394FF500500051280F405118095
:10F8B000E6051080D853903B43A03DD2954390C0BD
:10F8C0007F033185900F35E0FF3185900F36E0FFE3
:10F8D0003185900F37E0FF3185C2917514007515A1
:10F8E00000C3E51494F840022169E5156400700432
:10F8F000E51464406016E51564007004E514648046
:10F90000600AE515B40007E514B4C002B2917F00A7
:10F9100031858F13E5154514700AE5136402600400
:10F92000D2258045AE14AF158E168F17AE14AF15C5
:10F930008E188F1975B7A575B7F1438F01AE16AF45
:10F94000178F828E83E513F0538FFEAE18AF198F99
:10F95000828E83E493FFE5136F6004D225800A054D
:10F9600015E5157002051401E153903B43A03DD20B
:10F97000953025047F0280027F00319900C291C238
:10F980009043EF9022900F38EFF0C2FF900F38E0D5
:10F99000FF8FA330FFFDAFA322900F39EFF05390FC
:10F9A0003B43A03DD295C2A5900F39E0FF3185536E
:08F9B000903B43A03DD29522DB
:00000001FF
